:100000000C9446000C94FC000C9406010C94100116
:100010000C9434010C9445010C944F010C9459013B
:100020000C9463010C946D010C9477010C94810184
:100030000C948B010C9495010C949F010C94A901D4
:100040000C94F0010C9463000C9463000C94630016
:100050000C9463000C94FA010C9463000C946300FC
:100060000C9463000C9463000C9463000C94630084
:100070000C9463000C9463000C9463000C94630074
:100080000C9463000C9463000C94630011241FBE55
:10009000CFEFD0E1DEBFCDBF11E0A0E0B1E0EAECF0
:1000A000F0E100E00BBF02C007900D92AA3BB10740
:1000B000D9F712E0AAEBB1E001C01D92A73EB1074B
:1000C000E1F70C9404020C9400008091BA0188239B
:1000D00061F48FEF8093BA010E943A024FEF61E022
:1000E0008091C8010E94C302F7CF08951F93F8942E
:1000F0000E940E021FEF1ABB1BBB83EE87BB18BA10
:1001000014BB15BA11BA12BA12B813B88CEF809397
:1001100064001092650080B7886080BF8FE183BF64
:1001200082E081BF87B7826087BF1093D20281EFE0
:100130008FBD81E08EBD88EC8093D1028091D10289
:100140008BBD8091D10289BD8091D1028ABD809101
:10015000D10288BD89E185BD8DE783BD10928B00FA
:100160008FE080938A0085B3912F981B9BBB789476
:1001700088EB80936A0084E48ABF89B7806289BF74
:1001800089B78C6089BF0E94600380E38093C501BA
:100190008AE090E09093CD028093CC021092DF022F
:1001A0001093D2020E9438040E9465001F910895A6
:1001B0001F920F920FB60F9211242F933F934F93DC
:1001C0005F936F937F938F939F93AF93BF93EF93BF
:1001D000FF930E947600FF91EF91BF91AF919F91A5
:1001E0008F917F916F915F914F913F912F910F90E0
:1001F0000FBE0F901F9018951F920F920FB60F927F
:1002000011240F900FBE0F901F9018951F920F9200
:100210000FB60F9211240F900FBE0F901F901895DC
:100220001F920F920FB60F9211242F933F934F936B
:100230005F936F937F938F939F93AF93BF93EF934E
:10024000FF930E94A103FF91EF91BF91AF919F9106
:100250008F917F916F915F914F913F912F910F906F
:100260000FBE0F901F9018951F920F920FB60F920E
:1002700011248F938091BE018F5F8093BE018F9177
:100280000F900FBE0F901F9018951F920F920FB6F0
:100290000F9211240F900FBE0F901F9018951F9270
:1002A0000F920FB60F9211240F900FBE0F901F9058
:1002B00018951F920F920FB60F9211240F900FBE38
:1002C0000F901F9018951F920F920FB60F92112446
:1002D0000F900FBE0F901F9018951F920F920FB6A0
:1002E0000F9211240F900FBE0F901F9018951F9220
:1002F0000F920FB60F9211240F900FBE0F901F9008
:1003000018951F920F920FB60F9211240F900FBEE7
:100310000F901F9018951F920F920FB60F921124F5
:100320000F900FBE0F901F9018951F920F920FB64F
:100330000F9211240F900FBE0F901F9018951F92CF
:100340000F920FB60F9211240F900FBE0F901F90B7
:1003500018951F920F920FB60F9211242F933F936F
:100360004F935F936F937F938F939F93AF93BF93BD
:10037000EF93FF93809188008093BD018091CB0221
:100380009091BD01890F8093CB020E948C020E9444
:1003900084050E945C060E94D1040E9428030E94EA
:1003A00042020E94A9048091CF028F5F8093CF0206
:1003B0008091D3028F5F8093D3021092BE01FF9190
:1003C000EF91BF91AF919F918F917F916F915F91CD
:1003D0004F913F912F910F900FBE0F901F90189546
:1003E0001F920F920FB60F9211240F900FBE0F9015
:1003F0001F9018951F920F920FB60F9211240F9015
:100400000FBE0F901F901895CFEFD0E1DEBFCDBF8C
:100410000E94760080E090E00C9464081092CF0275
:100420001092D0021092BD011092BE018FEF809306
:10043000D1021092C9011092D8021092C3011092F9
:10044000CE021092BF011092D5021092D202809378
:10045000C1018093C2011092DB021092BC01109284
:10046000D9021092DE021092C8011092E40210929A
:10047000E60208958091DF02882319F48093D20266
:1004800086B9089585B38F709091C501892B85BB7E
:100490008091D1028A3018F48FEF8093D10280913D
:1004A000D1028BBD8091D10289BD8091D1028ABDDC
:1004B0008091D10288BD08958091C501803C91F062
:1004C00080EC8093C5011092CB021092D40210925E
:1004D000D3021092C9021092CE028FEF8093C30113
:1004E0000E9442028091CB028A3028F48091D3028C
:1004F0008E3128F408958091CB028093C902109226
:10050000CB021092D4021092D3021092C301109227
:10051000CE021092BF0108958091D5028150809340
:10052000D5028091D502883C28F18091630090919A
:1005300063009270969580FF0CC0913051F4109238
:10054000D5021092DB028FEF8093C1018093C2012C
:1005500008958FEF8093D5021092C1011092C201CD
:100560001092C5018EEF8093D10286E00E94E203D3
:100570000E94A90408951092C5018FEF8093D102C3
:100580000E94420208954F3F11F4481B4BBB08954F
:100590000E9407086AE00E94170897E0899F802D53
:1005A00011246DE20E941708880F880F880F992781
:1005B00008958091C501803C69F080EC8093C5016D
:1005C0001092CB021092D4021092D3021092C90260
:1005D0000E9442028091D402843028F48091D30298
:1005E000853028F408958091CB028093C90210923F
:1005F000CB021092D4021092D3021092CE0210922B
:10060000BF010E94C8028093E5028091E5020E942A
:10061000FF0608958091CC029091CD02181619061C
:100620002CF48091CC029091CD02F4CF089520E07B
:10063000281730F490E09F5F9F3FE9F72F5FF8CFD6
:1006400008958091C701882311F08150FCCF08954F
:100650001F93CF93DF93CDB7DEB726970FB6F894ED
:10066000DEBF0FBECDBFDE011196E0E0F1E086E017
:1006700001900D928150E1F71091C4011123B1F462
:100680008AE185BD898183BD85B38F6085BB14BD3B
:1006900084E08093C7010E94210313BD85B3807F4E
:1006A00085BB82E08093C7010E94210326960FB686
:1006B000F894DEBF0FBECDBFDF91CF911F9108959B
:1006C000CF93DF93CDB7DEB72A970FB6F894DEBF8E
:1006D0000FBECDBF9E012F5F3F4FD901E6E0F1E095
:1006E0009AE001900D929150E1F78AE08093D60252
:1006F0009093DA029091DA028091D602981798F4DA
:100700008091DA02A82FBB27A653BE4F8091DA0250
:10071000F901E80FF11D80818C938091DA028F5FDF
:100720008093DA02E7CF1092C6018FEF8093DD024B
:100730002A960FB6F894DEBF0FBECDBFDF91CF91E2
:100740000895CF93DF93CDB7DEB728970FB6F8940F
:10075000DEBF0FBECDBF9E012F5F3F4FD901E0E14D
:10076000F1E098E001900D929150E1F788E08093DC
:10077000D6029093DA029091DA028091D60298170D
:1007800098F48091DA02A82FBB27A653BE4F809120
:10079000DA02F901E80FF11D80818C938091DA0271
:1007A0008F5F8093DA02E7CF1092C6018FEF8093BC
:1007B000DD0228960FB6F894DEBF0FBECDBFDF91E5
:1007C000CF910895CF93DF93CDB7DEB7C356D04016
:1007D0000FB6F894DEBF0FBECDBF282FAE014F5F1E
:1007E0005F4FDA01E8E1F1E093E601900D9291505C
:1007F000E1F78BE08093D6029093DA029091DA02CF
:100800008091D602981728F533278BE090E0289F37
:10081000B001299F700D389F700D11249B018091AC
:10082000DA02A82FBB27A653BE4F8091DA02F90146
:10083000E80FF11DE40FF51F80818C938091DA029F
:100840008F5F8093DA029091DA028091D602981736
:1008500030F31092C6018FEF8093DD02CD59DF4F48
:100860000FB6F894DEBF0FBECDBFDF91CF910895D4
:1008700089E18093D60281E08093DA029091DA02D6
:100880008091D602981768F48091DA02E82FFF274A
:10089000E653FE4F8091DA0280838091DA028F5F07
:1008A000EBCF1092C6018FEF8093DD020895CF93B6
:1008B000DF93CDB7DEB7AA970FB6F894DEBF0FBEB1
:1008C000CDBFAE014F5F5F4FCA012BE731E0AAE217
:1008D000F90101909F01FC010192CF01A150C1F7E4
:1008E0002A2F8AE28093D602A093DA029091DA024C
:1008F0008091D6029817F8F43FEFA22FBB27A6539A
:10090000BE4F8091DA02FA01E80FF11D8081845F09
:100910008C932F5FE22FFF27E653FE4F30832F5F2C
:100920008091DA028F5F8093DA029091DA028091EF
:10093000D602981710F31092C6018FEF8093DD0254
:10094000AA960FB6F894DEBF0FBECDBFDF91CF9150
:1009500008958091DD028F3F19F58091C601E82F3F
:10096000FF27E653FE4FE0818091C6018F5F8093A1
:10097000C601EE2399F080E0EF3F09F08DE185BDDF
:10098000E3BD85B38093DA028091DA02807F825FD3
:100990008093DA028091DA0285BB0895E093DD024C
:1009A0000895EF92FF920F931F93CF93DF93CDB7EC
:1009B000DEB760970FB6F894DEBF0FBECDBF7E01E5
:1009C0000894E11CF11CD701E5EAF1E090E1019007
:1009D0000D929150E1F78091DB028F3F09F487C0BF
:1009E00011E08AE185BD898183BD012F9093BC010F
:1009F0009093D90285B38093E2028091E202807FD6
:100A00008093E2028091E20285BB8091E2028F5FD7
:100A10008093E20282E00E94170382E00E941703A3
:100A200082E00E9417030C9905C08091BC01812BC4
:100A30008093BC01F701E00FF11D808183BD0F5F42
:100A400085B3807F85BB82E00E94170382E00E940D
:100A5000170382E00E941703110F59F48091D90205
:100A6000882321F48091BC018093D9021093BC01AA
:100A700011E00E3038F28091BC018093DE021092BA
:100A8000C8018091D90281FF05C08091C8018160B1
:100A90008093C8018091D90282FF05C08091C8016E
:100AA00080618093C8018091D90283FF05C0809145
:100AB000C80180648093C8018091D90284FF05C079
:100AC0008091C80182608093C8018091D90285FF1E
:100AD00005C08091C80188608093C8018091D902C7
:100AE00086FF05C08091C80180688093C801609628
:100AF0000FB6F894DEBF0FBECDBFDF91CF911F912F
:100B00000F91FF90EF900895CF938091C1018F3F97
:100B100009F0D0C0C82F8091C8018178813851F088
:100B20000E94D1048091C8018178813819F00E9417
:100B30005C02C0E08091E402882389F0CF3F79F421
:100B40008091C8018A7519F48093E40208C0C0E05E
:100B500084E00E94E2038091E5020E94FF068091FA
:100B6000E602882369F0CF3F59F48091C8018A7565
:100B700019F48093E60207C085E00E94E20318C0E2
:100B8000CF3F09F097C08091C9018F3F49F40E947F
:100B9000C8028093E5028091E5020E94FF068AC0A8
:100BA0008091D8028F3F49F40E94C8028093E502E9
:100BB0008091E5020E9436077DC08091C3018F3F7E
:100BC00021F08091CE028F3F19F40E945C0272C026
:100BD0008091BF01883C18F00E94D9026BC08091BF
:100BE000D2028F3F19F40E94BB0264C08091C801F9
:100BF0008A7529F58091C501992780339105D9F02F
:100C0000813391051CF4892B69F003C0803C910568
:100C100041F18091D1028A3A28F48091D1028E5C10
:100C20008093D1028091D102883C28F48091D10236
:100C3000825E8093D10280E38093C5013BC00E9415
:100C400060038091C80181FD04C08091C80186FFC6
:100C500014C08091C501803969F08091C50180364A
:100C600049F08091D102883228F08091D1028A51D6
:100C70008093D1020E946D071DC08091C501992704
:100C80008033910591F0813391051CF4892B69F033
:100C900003C0803C910549F08091D1028A3A28F442
:100CA0008091D1028E5C8093D10280EC8093C5014B
:100CB0000E944202CF9108951F938091C2018F3FFD
:100CC00009F09BC08091BD01833060F08091BE012E
:100CD000882319F01092BF0105C08091BF018C5E7E
:100CE0008093BF01109288008091CC029091CD0238
:100CF00001979093CD028093CC028091CF028823FC
:100D000021F48CED8093D10275C09091CF02809137
:100D1000D002981708F471C01092CF029091BD01D3
:100D20009923A1F48091D102883220F08091D102E0
:100D300084515CC08FEF8093CE0288EC8093D10207
:100D400083E08093D0029093CF0257C08091BD0181
:100D5000823008F441C08091BD01843008F44DC058
:100D60008091BD01863080F18091BD01883010F105
:100D70008091BD018A30D0F08091BD01843158F05E
:100D80001092CF021092C50180EF8093D10282E0D1
:100D90008093D0022DC01091C5011092C5018EE044
:100DA0000E9417031093C50188EF20C08091D102E3
:100DB000885D15C08091D1028C5E8093D1028091B4
:100DC000D1028431A8F411C08091D102803F80F417
:100DD0008091D1028B5F0AC08091D10285508093AF
:100DE000D1028091D102883218F480EF8093D10231
:100DF0001092CF0283E08093D0021F910895CF9389
:100E0000CFEF8091C501803969F080E98093C501F9
:100E10001092CB021092D3021092C9020E94420299
:100E2000C093C9019091CB028091E502981728F0F8
:100E30008091CB028093C902C0E08091D302282F19
:100E400033279091E50283E0989FC0011124281771
:100E5000390714F4CC2341F41092CB021092C9014B
:100E60001092D3021092E002CF910895CF93CFEF6A
:100E70008091C501803669F080E68093C5011092AB
:100E8000CB021092D3021092C9020E944202C09378
:100E9000D8029091CB028091E502981728F08091BA
:100EA000CB028093C902C0E08091D302282F332760
:100EB0009091E50283E0989FC0011124281739071B
:100EC00014F4CC2341F41092CB021092D802109269
:100ED000D3021092E002CF9108950E9407088093F8
:100EE000E3022091E30221708091E302992782704E
:100EF000907095958795813079F48091E3028471A3
:100F00008093E502213021F48FEF8093E60209C03F
:100F10008FEF8093E40205C08091E3028A7580938D
:100F2000E5028091E502853018F485E08093E502C2
:100F3000213029F48091E5020E94360708958091BE
:100F4000E5020E94FF060895AF92BF92CF92DF9212
:100F5000EF92FF920F931F93CF93DF93EC01E88002
:100F6000F9800A811B81C801B7012DE133EF41E00F
:100F700050E00E94420859016A01C801B7012DE101
:100F800033EF41E050E00E944208DC01CB01BC019C
:100F9000CD0127EA31E440E050E00E9423087B01C4
:100FA0008C01C601B50124E13BE040E050E00E9425
:100FB0002308DC01CB01E81AF90A0A0B1B0B1E14EB
:100FC0001F041006110644F08FEF9FEFAFEFBFE74D
:100FD000E80EF91E0A1F1B1FE882F9820A831B8391
:100FE0008FEF9FE7A0E0B0E0E822F9220A231B235D
:100FF000C701DF91CF911F910F91FF90EF90DF908C
:10100000CF90BF90AF9008950E94A407089585EBFC
:1010100091E00E94A4070895AA27BB278093B501F9
:101020009093B601A093B701B093B8010895991BAE
:1010300079E004C0991F961708F0961B881F7A95CF
:10104000C9F780950895629FD001739FF001829F38
:10105000E00DF11D649FE00DF11D929FF00D839F47
:10106000F00D749FF00D659FF00D9927729FB00DE4
:10107000E11DF91F639FB00DE11DF91FBD01CF01F7
:1010800011240895A1E21A2EAA1BBB1BFD010DC05D
:10109000AA1FBB1FEE1FFF1FA217B307E407F50728
:1010A00020F0A21BB30BE40BF50B661F771F881F04
:1010B000991F1A9469F760957095809590959B019A
:0A10C000AC01BD01CF010895FFCF80
:1010CA00181818181818140F0A05140F0A05000022
:1010DA000F1996640FC81400050A0F141919140F72
:1010EA000A0500196419641964196419640005056C
:1010FA00190505190505191900C8C8FFC8C8FFC888
:10110A00C8FFFF00C8FFC8FFC8FF0000000000F0CA
:10111A00FFF0FFF0FF00000000006464FF6464FF5A
:10112A006464FF64000DFF14FF0DFF14FF0DFF0040
:10113A0001FF02FF03FF04FF05FF000AFF050A057E
:10114A000A050A0DFF0A0D0A0D0A0D11FF0D110FEE
:10115A00FF0C0F0DFF0A0D0CFF11FF1110100D0DE2
:10116A000C0C0A0AFF2C181C18181C181818181826
:0A117A00181818180001000000000A
:00000001FF
